Stack Allocation = 8192 bytes

 wowexec

 Start     Length     Name                   Class
 0001:0000 011B9H     _TEXT                  CODE
 0001:11BA 00276H     _COMMAND               CODE
 0002:0000 00010H     NULL                   BEGDATA
 0002:0010 000DCH     _DATA                  DATA
 0002:00EC 00000H     CDATA                  DATA
 0002:00EC 00000H     XIFB                   DATA
 0002:00EC 00000H     XIF                    DATA
 0002:00EC 00000H     XIFE                   DATA
 0002:00EC 00000H     XIB                    DATA
 0002:00EC 00000H     XI                     DATA
 0002:00EC 00000H     XIE                    DATA
 0002:00EC 00000H     XPB                    DATA
 0002:00EC 00000H     XP                     DATA
 0002:00EC 00000H     XPE                    DATA
 0002:00EC 00000H     XCB                    DATA
 0002:00EC 00000H     XC                     DATA
 0002:00EC 00000H     XCE                    DATA
 0002:00EC 00000H     XCFB                   DATA
 0002:00EC 00000H     XCF                    DATA
 0002:00EC 00000H     XCFE                   DATA
 0002:00EC 0000CH     DBDATA                 DATA
 0002:00F8 00000H     CONST                  CONST
 0002:0100 00000H     _BSS                   BSS
 0002:0100 00000H     XOB                    BSS
 0002:0100 00000H     XO                     BSS
 0002:0100 00000H     XOE                    BSS
 0002:0100 0018BH     c_common               BSS

 Origin   Group
 0002:0   DGROUP

 Address   Export                  Alias

 0001:0BD2 FaxWndProc              FaxWndProc
 0001:0908 WndProc                 WndProc

  Address         Publics by Name

 0000:0000  Imp  ANSITOOEM            (KEYBOARD.5)
 0000:0000  Imp  BRINGWINDOWTOTOP     (USER.45)
 0000:0000  Imp  CREATEWINDOW         (USER.41)
 0000:0000  Imp  DEFWINDOWPROC        (USER.107)
 0000:0000  Imp  DISPATCHMESSAGE      (USER.114)
 0000:0000  Imp  DOS3CALL             (KERNEL.102)
 0001:1350       DOSDELETE
 0001:1387       DOSRENAME
 0000:0000  Imp  ENUMWINDOWS          (USER.54)
 0001:02AA       EXECAPPLICATION
 0001:0150       EXECPROGRAM
 0001:0BD2       FaxWndProc
 0001:1201       FILETIME
 0001:009A       FINDPOPUPFROMEXE
 0001:0010       FINDPREVINSTANCEPROC
 0000:0000  Imp  FINDWINDOW           (USER.50)
 0000:0000  Imp  FREELIBRARY          (KERNEL.96)
 0001:12C5       GETCURRENTDIRECTORY
 0001:128C       GETCURRENTDRIVE
 0000:0000  Imp  GETCURRENTTASK       (KERNEL.36)
 0001:1266       GETDOSERRORCODE
 0001:09EE       GETFILENAMEFROMPATH
 0000:0000  Imp  GETLASTACTIVEPOPUP   (USER.287)
 0000:0000  Imp  GETMODULEFILENAME    (KERNEL.49)
 0000:0000  Imp  GETPARENT            (USER.46)
 0001:0A26       GETPATHINFO
 0000:0000  Imp  GETPRIVATEPROFILESTRING (KERNEL.128)
 0000:0000  Imp  GETPROCADDRESS       (KERNEL.50)
 0000:0000  Imp  GETSTOCKOBJECT       (GDI.87)
 0000:0000  Imp  GETSYSTEMMETRICS     (USER.179)
 0000:0000  Imp  GETWINDOW            (USER.262)
 0000:0000  Imp  GETWINDOWSDIRECTORY  (KERNEL.134)
 0000:0000  Imp  GETWINDOWTASK        (USER.224)
 0000:0000  Imp  GETWINDOWWORD        (USER.133)
 0000:0000  Imp  GLOBALALLOC          (KERNEL.15)
 0000:0000  Imp  GLOBALDELETEATOM     (USER.269)
 0000:0000  Imp  GLOBALFREE           (KERNEL.17)
 0000:0000  Imp  GLOBALGETATOMNAME    (USER.271)
 0000:0000  Imp  GLOBALLOCK           (KERNEL.18)
 0000:0000  Imp  GLOBALUNLOCK         (KERNEL.19)
 0000:0000  Imp  INITAPP              (USER.5)
 0000:0000  Imp  INITTASK             (KERNEL.91)
 0000:0000  Imp  ISICONIC             (USER.31)
 0001:1229       ISREADONLY
 0000:0000  Imp  ISWINDOWENABLED      (USER.35)
 0000:0000  Imp  ISWINDOWVISIBLE      (USER.49)
 0001:13D7       LMEMMOVE
 0000:0000  Imp  LOADCURSOR           (USER.173)
 0000:0000  Imp  LOADICON             (USER.174)
 0000:0000  Imp  LOADLIBRARY          (KERNEL.95)
 0000:0000  Imp  LOADMODULE           (KERNEL.45)
 0000:0000  Imp  LOADSTRING           (USER.176)
 0000:0000  Imp  LOCKSEGMENT          (KERNEL.23)
 0000:0000  Imp  LSTRCAT              (KERNEL.89)
 0000:0000  Imp  LSTRCMPI             (USER.471)
 0000:0000  Imp  LSTRCPY              (KERNEL.88)
 0000:0000  Imp  LSTRLEN              (KERNEL.90)
 0001:0584       MYMESSAGEBOX
 0000:0000  Imp  OPENDRIVER           (USER.252)
 0000:0000  Imp  OUTPUTDEBUGSTRING    (KERNEL.115)
 0001:09D8       PARTYDIALOGPROC
 0001:11BA       PATHTYPE
 0000:0008  Abs  pAtomTable
 0000:0000  Imp  PEEKMESSAGE          (USER.109)
 0000:0006  Abs  pLocalHeap
 0000:000E  Abs  pStackBot
 0000:000C  Abs  pStackMin
 0000:000A  Abs  pStackTop
 0000:0000  Imp  REGISTERCLASS        (USER.57)
 0002:0004       rsrvptrs
 0001:130E       SETCURRENTDIRECTORY
 0001:12A6       SETCURRENTDRIVE
 0000:0000  Imp  SHOWCURSOR           (USER.71)
 0000:0000  Imp  SHOWWINDOW           (USER.42)
 0001:0AB2       STARTREQUESTEDAPP
 0002:00E0       STKHQQ
 0000:0000  Imp  TRANSLATEMESSAGE     (USER.113)
 0000:0000  Imp  UNLOCKSEGMENT        (KERNEL.24)
 0000:0000  Imp  WAITEVENT            (KERNEL.30)
 0000:0000  Imp  WINEXEC              (KERNEL.166)
 0001:0650       WINMAIN
 0001:0908       WndProc
 0000:0000  Imp  WOWFAILEDEXEC        (KERNEL.508)
 0000:0000  Imp  WOWGETNEXTVDMCOMMAND (KERNEL.502)
 0000:0000  Imp  WOWMSGBOX            (KERNEL.263)
 0000:0000  Imp  WOWPARTYBYNUMBER     (KERNEL.273)
 0000:0000  Imp  WOWQUERYDEBUG        (KERNEL.512)
 0000:0000  Imp  WOWREGISTERSHELLWINDOWHANDLE (KERNEL.503)
 0000:0000  Imp  WOWSETEXITONLASTAPP  (KERNEL.541)
 0000:0000  Imp  WOWWAITFORMSGANDEVENT (KERNEL.262)
 0001:00EE       _ActivatePrevInstance
 0002:0100       _edata
 0002:028B       _end
 0001:1143       _exit
 0001:10AE       _FaxInit
 0002:0018       _gfSharedWOW
 0002:0012       _ghwndEdit
 0002:0010       _ghwndMain
 0002:0182       _gwFirstCmdShow
 0002:0206       _hAppInstance
 0001:07CE       _InitializeApp
 0002:0014       _lpszAppTitle
 0002:024A       _szAppTitleBuffer
 0002:0208       _szOOMExitMsg
 0002:026A       _szOOMExitTitle
 0002:0184       _szOriginalDirectory
 0002:0100       _szWindowsDirectory
 0000:0000  Imp  _wsprintf            (USER.420)
 0000:9876  Abs  __acrtused
 0000:9876  Abs  __acrtused2
 0000:D6D6  Abs  __aDBdoswp
 0002:00F0       __aDBrterr
 0001:1159       __astart
 0002:0100       __edata
 0002:028B       __end
 0001:1143       __exit
 0000:9876  Abs  __fptaskdata
 0001:1141       __wflags
 0000:0000  Imp  __WINFLAGS           (KERNEL.178)
 0002:00F2       ___aDBexit
 0002:00EE       ___aDBswpchk
 0002:00EC       ___aDBswpflg

  Address         Publics by Value

 0000:0000  Imp  GETLASTACTIVEPOPUP   (USER.287)
 0000:0000  Imp  GLOBALFREE           (KERNEL.17)
 0000:0000  Imp  ENUMWINDOWS          (USER.54)
 0000:0000  Imp  GETPARENT            (USER.46)
 0000:0000  Imp  DISPATCHMESSAGE      (USER.114)
 0000:0000  Imp  WOWPARTYBYNUMBER     (KERNEL.273)
 0000:0000  Imp  GETSYSTEMMETRICS     (USER.179)
 0000:0000  Imp  DOS3CALL             (KERNEL.102)
 0000:0000  Imp  REGISTERCLASS        (USER.57)
 0000:0000  Imp  LOADICON             (USER.174)
 0000:0000  Imp  ISICONIC             (USER.31)
 0000:0000  Imp  __WINFLAGS           (KERNEL.178)
 0000:0000  Imp  WOWWAITFORMSGANDEVENT (KERNEL.262)
 0000:0000  Imp  GETPRIVATEPROFILESTRING (KERNEL.128)
 0000:0000  Imp  UNLOCKSEGMENT        (KERNEL.24)
 0000:0000  Imp  WOWQUERYDEBUG        (KERNEL.512)
 0000:0000  Imp  WINEXEC              (KERNEL.166)
 0000:0000  Imp  LOADCURSOR           (USER.173)
 0000:0000  Imp  WOWREGISTERSHELLWINDOWHANDLE (KERNEL.503)
 0000:0000  Imp  GETWINDOWWORD        (USER.133)
 0000:0000  Imp  PEEKMESSAGE          (USER.109)
 0000:0000  Imp  ISWINDOWVISIBLE      (USER.49)
 0000:0000  Imp  GLOBALUNLOCK         (KERNEL.19)
 0000:0000  Imp  WOWSETEXITONLASTAPP  (KERNEL.541)
 0000:0000  Imp  GETCURRENTTASK       (KERNEL.36)
 0000:0000  Imp  BRINGWINDOWTOTOP     (USER.45)
 0000:0000  Imp  GLOBALLOCK           (KERNEL.18)
 0000:0000  Imp  WOWFAILEDEXEC        (KERNEL.508)
 0000:0000  Imp  LOADLIBRARY          (KERNEL.95)
 0000:0000  Imp  GETWINDOWTASK        (USER.224)
 0000:0000  Imp  _wsprintf            (USER.420)
 0000:0000  Imp  OPENDRIVER           (USER.252)
 0000:0000  Imp  LSTRLEN              (KERNEL.90)
 0000:0000  Imp  WAITEVENT            (KERNEL.30)
 0000:0000  Imp  TRANSLATEMESSAGE     (USER.113)
 0000:0000  Imp  FREELIBRARY          (KERNEL.96)
 0000:0000  Imp  INITAPP              (USER.5)
 0000:0000  Imp  GETWINDOWSDIRECTORY  (KERNEL.134)
 0000:0000  Imp  LOCKSEGMENT          (KERNEL.23)
 0000:0000  Imp  GETSTOCKOBJECT       (GDI.87)
 0000:0000  Imp  WOWMSGBOX            (KERNEL.263)
 0000:0000  Imp  OUTPUTDEBUGSTRING    (KERNEL.115)
 0000:0000  Imp  WOWGETNEXTVDMCOMMAND (KERNEL.502)
 0000:0000  Imp  GETWINDOW            (USER.262)
 0000:0000  Imp  GETPROCADDRESS       (KERNEL.50)
 0000:0000  Imp  LSTRCAT              (KERNEL.89)
 0000:0000  Imp  LSTRCPY              (KERNEL.88)
 0000:0000  Imp  GLOBALALLOC          (KERNEL.15)
 0000:0000  Imp  CREATEWINDOW         (USER.41)
 0000:0000  Imp  GETMODULEFILENAME    (KERNEL.49)
 0000:0000  Imp  SHOWCURSOR           (USER.71)
 0000:0000  Imp  ISWINDOWENABLED      (USER.35)
 0000:0000  Imp  LOADSTRING           (USER.176)
 0000:0000  Imp  ANSITOOEM            (KEYBOARD.5)
 0000:0000  Imp  INITTASK             (KERNEL.91)
 0000:0000  Imp  FINDWINDOW           (USER.50)
 0000:0000  Imp  GLOBALGETATOMNAME    (USER.271)
 0000:0000  Imp  DEFWINDOWPROC        (USER.107)
 0000:0000  Imp  LOADMODULE           (KERNEL.45)
 0000:0000  Imp  GLOBALDELETEATOM     (USER.269)
 0000:0000  Imp  LSTRCMPI             (USER.471)
 0000:0000  Imp  SHOWWINDOW           (USER.42)
 0000:0006  Abs  pLocalHeap
 0000:0008  Abs  pAtomTable
 0000:000A  Abs  pStackTop
 0000:000C  Abs  pStackMin
 0000:000E  Abs  pStackBot
 0000:9876  Abs  __acrtused2
 0000:9876  Abs  __acrtused
 0000:9876  Abs  __fptaskdata
 0000:D6D6  Abs  __aDBdoswp
 0001:0010       FINDPREVINSTANCEPROC
 0001:009A       FINDPOPUPFROMEXE
 0001:00EE       _ActivatePrevInstance
 0001:0150       EXECPROGRAM
 0001:02AA       EXECAPPLICATION
 0001:0584       MYMESSAGEBOX
 0001:0650       WINMAIN
 0001:07CE       _InitializeApp
 0001:0908       WndProc
 0001:09D8       PARTYDIALOGPROC
 0001:09EE       GETFILENAMEFROMPATH
 0001:0A26       GETPATHINFO
 0001:0AB2       STARTREQUESTEDAPP
 0001:0BD2       FaxWndProc
 0001:10AE       _FaxInit
 0001:1141       __wflags
 0001:1143       _exit
 0001:1143       __exit
 0001:1159       __astart
 0001:11BA       PATHTYPE
 0001:1201       FILETIME
 0001:1229       ISREADONLY
 0001:1266       GETDOSERRORCODE
 0001:128C       GETCURRENTDRIVE
 0001:12A6       SETCURRENTDRIVE
 0001:12C5       GETCURRENTDIRECTORY
 0001:130E       SETCURRENTDIRECTORY
 0001:1350       DOSDELETE
 0001:1387       DOSRENAME
 0001:13D7       LMEMMOVE
 0002:0004       rsrvptrs
 0002:0010       _ghwndMain
 0002:0012       _ghwndEdit
 0002:0014       _lpszAppTitle
 0002:0018       _gfSharedWOW
 0002:00E0       STKHQQ
 0002:00EC       ___aDBswpflg
 0002:00EE       ___aDBswpchk
 0002:00F0       __aDBrterr
 0002:00F2       ___aDBexit
 0002:0100       __edata
 0002:0100       _szWindowsDirectory
 0002:0100       _edata
 0002:0182       _gwFirstCmdShow
 0002:0184       _szOriginalDirectory
 0002:0206       _hAppInstance
 0002:0208       _szOOMExitMsg
 0002:024A       _szAppTitleBuffer
 0002:026A       _szOOMExitTitle
 0002:028B       _end
 0002:028B       __end

Program entry point at 0001:1159
